:040000006F3070628B
:1000040000000000000000004A3B00006A3B0000C2
:1000140000000000243E000000000000000000007A
:10002400243E0000243E0000000000000000000008
:10003400A232000000000000900200000000000056
:10004400243E0000243E0000243E0000243E000024
:10005400243E0000243E00000A370000323700002E
:100064005A37000082370000AA370000243E0000FF
:10007400243E0000243E0000243E0000243E0000F4
:10008400243E0000243E0000243E0000243E0000E4
:10009400243E0000243E0000243E0000D23700002D
:1000A400243E0000243E0000243E0000243E0000C4
:1000B400243E0000243E0000243E0000243E0000B4
:1000C400243E0000243E0000243E0000243E0000A4
:1000D400243E0000003B0000243E0000D44B0000FE
:1000E4004A380000243E0000243E0000243E000064
:1000F400243E0000243E0000243E0000243E000074
:1001040000000000243E0000243E0000243E0000C5
:10011400243E0000243E0000243E0000243E000053
:10012400243E0000243E0000243E0000243E000043
:10013400243E0000243E0000243E0000243E000033
:10014400243E0000243E0000243E0000243E000023
:10015400243E0000243E0000243E0000243E000013
:10016400243E0000243E0000243E0000243E000003
:10017400243E0000243E0000243E0000243E0000F3
:10018400243E0000243E0000243E0000243E0000E3
:10019400243E0000243E0000243E0000243E0000D3
:1001A400000000000000000000000000000000004B
:0C01B4000000000000000000000000003F
:1001C00097020120938202E4938202E0739002344A
:1001D00003210500224573100530B1A819712320B1
:1001E000250006C006C216CAF322003093F2820030
:1001F000638402009302000816C412C81ACC1ECEF3
:1002000022D026D22AD42ED632D836DA3ADC3EDEB6
:10021000C2C0C6C2CAC4CEC6D2C8D6CADACCDECE26
:10022000E2D0E6D2EAD4EED6F2D8F6DAFADCFEDE96
:1002300003A1050009A002457310153492403785CB
:10024000000013050580732005302245732005301A
:100250004242D2426243F243025492542255B25572
:100260004256D2566257F257064896482649B64932
:10027000464AD64A664BF64B065C965C265DB65DF2
:10028000465ED65E665FF65F09617300203000004F
:10029000197116CA9302000816C49302000273A0D3
:1002A000428006C212C81ACC1ECE22D026D22AD430
:1002B0002ED632D836DA3ADC3EDEC2C0C6C2CAC456
:1002C000CEC6D2C8D6CADACCDECEE2D0E6D2EAD4E6
:1002D000EED6F2D8F6DAFADCFEDE73110134EF0066
:1002E000F006EF10703AEF005009731101341384D7
:1002F0008189032904006304090223200400732573
:1003000010342AC013840189044023A024001384DC
:100310004189044003A10400024573101534924042
:10032000B78200009382028073A00230A24273A0C1
:1003300002304242D2426243F24302549254225566
:10034000B2554256D2566257F25706489648264949
:10035000B649464AD64A664BF64B065C965C265D25
:10036000B65D465ED65E665FF65F0961730020305B
:100370000000397101436EC619A0397141536AC832
:1003800066CA62CC5ECE19A0397101535AD056D2DA
:1003900052D44ED64AD826DA22DC06DE330161403A
:1003A000828241114AC026C222C406C68282B24D50
:1003B0004101024D924C224CB24B4101024B924AF8
:1003C000224AB2494101024992442244B2404101C9
:1003D00082803D432A876373C3029377F700BDEFA2
:1003E000ADE5937606FF3D8ABA960CC34CC30CC7A5
:1003F0004CC74107E36BD7FE11E28280B306C340CE
:100400008A069702000096966780A6002307B70029
:10041000A306B7002306B700A305B7002305B7005E
:10042000A304B7002304B700A303B7002303B70056
:10043000A302B7002302B700A301B7002301B7004E
:10044000A300B7002300B700828093F5F50F9396C1
:100450008500D58D93960501D58D61B793962700BC
:100460009702000096968682E78086FA9680C117EA
:100470001D8F3E96E374C3F8A5B703A581808280E3
:10048000EFF23FF2938781809843050798C3EF10FE
:10049000E0623C45FD173CC589E77C413CC5EF1057
:1004A000A066EF10D01105B7634205029307803EA6
:1004B0003347F5023365F5023305F5021305753E42
:1004C0003345F5023307F7023A9582807D558280E5
:1004D00001458280014582800145828001458280FC
:1004E000EFF23FEC196499641304847693844477A3
:1004F00063639400C9BD1C4011048297D5BFEFF21D
:100500005FEA19649964130444779384C47763633E
:10051000940055BD1C4011048297D5BFEFF27FE8CF
:10052000F93FEF30806645B5EFF2BFE7B705000051
:1005300037550000D14715479306002001469385A3
:10054000C5511305850DEF10C057EF10406FA5BDC5
:10055000EFF23FE5EF103014EF20504DEF00905CCC
:10056000EF10700DEF102029C137EF10700D192C0E
:10057000EF10402B014581BDEFF2BFE2D13F0145B5
:1005800099B5EFF27FE0AA89EF10405319C1EF103F
:10059000603B2545EF10C0114441130445006396AC
:1005A0008400EF10A051014919A8138944FF214686
:1005B000CE854A85EF00301401E9EF10205019C1B3
:1005C000EF10A0394A85DDBB8440D1BF09E57D55D8
:1005D00082807D55CDBBEFF2DFDC2A842E85328907
:1005E000AE8445377DF522852686A545EF10E00EC1
:1005F0000145231C2401230E0400231D0400D9BF40
:10060000EFF23FDA1E2D41112A84C18B9DE71C5564
:100610008DC32EC68297AA84B24501CD2A8637554E
:100620000000A2851305050EEF0050492685410103
:1006300059BB1E2C93E707011EAC1E2CA18B89C74A
:100640003E2CE554A18BFDF35C5489CF2285829723
:10065000AA8405E13E2C93E787003EAC5C2C85071D
:100660005CACE9B785679387F7F0FD8D2EAC8144CC
:10067000D5B7E957E31CF5FAF1BF5C2D85CBEFF256
:100680005FD2FD1793F7F70F5CAD2A84014789EF1E
:100690001C5989E70147231D040039A082972A8746
:1006A00075D9E957E309F5FE3A8531BB7D573A859F
:1006B0008280EFF21FCF582D11E77D55EF000067C4
:1006C000014521A05C5999C38297F5B96955FDB7D9
:1006D000EFF23FCD582D11E77D55EF002065014524
:1006E00021A01C5D99C38297F9B96955FDB70CD15A
:1006F00001458280EFF25FC993894186854A83A7CD
:10070000418663863705EF10007983A741862A8AE0
:10071000638D370303A441865C4018401309C4FE6F
:100720005CC398C340C000C0EF10C0217C5099C387
:100730004A8582974A85EF10800B631B55014A85D5
:10074000EF00907FEF1060215285EF108075BDB1F2
:10075000EF10A0205285EF10C0744848EF00B06A37
:100760004A85EF10A00561BFEFF2BFC31384419526
:10077000130904011C4091C382971104E31C24FF58
:10078000953FEDB7EFF2FFC137060000B755000007
:10079000930800023D489307002013874196814645
:1007A00013068676938585111385418DEF10E02D14
:1007B0001385418DEF10A04839B1EFF29FBE2A8416
:1007C000FD541C406314F4000145F5BEEF10A06C0D
:1007D0002A89084044CD3115EF10A0414A85EF1019
:1007E000406CC5B7EFF2FFBB41112A842E8532C69B
:1007F0002EC4EF1080363246A24519C68547630DD8
:10080000F60001454101C1B65840938745011CC31C
:1008100098CD5CC0C0C9F5B71C406388870083C60B
:10082000550303C7170263FAE600D4431387450153
:1008300098C294CDD8C3DCC9E9B79C43F9BFEFF2A5
:100840005FB64111B2842E8689452A8436C6EF00F0
:10085000D068B246930744011CCC5CC846AC14B4C3
:10086000014541018DB6EFF23FB283A701854111E9
:100870002EC62A8491C38297EF10E0615E2CAA896C
:1008800089CFFD175EACEF10C06183A7C18401451D
:1008900091CB22858297014531A0B24791E7EF10B5
:1008A00040607955410119BEEF104021232805020F
:1008B0001034AA85AA84130544012D37B247635C1E
:1008C000F0001389C404700081454A85EF10A04BE5
:1008D0004A85EF1020404E85EF10A05CEF00507766
:1008E000885845D5C1B7EFF2DFAB83A781842A844E
:1008F00091C38297EF10205AAA8448489307440175
:10090000630EF5003115EF10C02E05442685EF105B
:10091000405919C0EF00D073014575B45E2C8507AE
:100920005EAC0144E5B7EFF2DFA72A8451057135CB
:10093000484CEF00504D2285EF005068014561B4EE
:10094000EFF23FA64111AE84AA85194532C636C4DE
:10095000EF0070612A841DC9A246930745011CCD92
:1009600014B55CC932461385340071994205418142
:1009700032B042060AB0418211053305C502EF00CC
:10098000903348CC19E52285793F01442285410105
:100990001DBC36302324040223260402232804022B
:1009A00001476345D70023120402CDB71E3010580B
:1009B0009107B387E7020507AA9790C31CD8D5B75C
:1009C0001E3163EEC706EFF23F9C83A781842A8421
:1009D0003289AE8991C38297EF10E04B045891E4BD
:1009E000EF10204C75556FF07F9D9C401CD8EF1088
:1009F000404B4A86CE8523A0040013854400C92EAF
:100A0000EF1060495C542A8991C384C31C5444D4B8
:100A100091E304D45E304848510485071EA8630C56
:100A200085003115EF10E01C4A85EF108047EF007C
:100A3000306201454DBF4A85EF10A046DDBF7D55B0
:100A40008280EFF29F9341112A842E8B328A36C620
:100A5000EF10C00683A701852A8999C32285829752
:100A6000EF1060435E30AA89639C070CB247814453
:100A70006399070CEF10E042795541016FF07F93C5
:100A8000B2472328090281EB4E85EF108041F957C8
:100A90002328F902D5B71034CA855E85A133B24741
:100AA000635DF000EFF07F9DAA847000814556855C
:100AB000EF10602D5685EF10E0214E85EF10603E5F
:100AC000EF001059032509034DF9EF10C03CB24760
:100AD000AA89268C635DF000EFF03F9AB247330C91
:100AE0009540A6973385A740634A05042AC6E28449
:100AF0005E30D9D70454984018D4585463149700E2
:100B000023260402FD175EB04E85EF1080391230A7
:100B10006373CA005286938544005A85552CEF10A2
:100B200080371C589CC004D8EF10A03783A7C1841D
:100B30000145A1D722858297014581B702C645BFED
:100B40008144930B4401930AC9045DB7EFF27F859A
:100B50004111EF104034138741811C23850793F71F
:100B6000F70F1CA383A7C18081C72AC6829732458D
:100B7000EF10203341016FF01F85EFF29F8241118A
:100B8000EF106031138741811C23FD1793F7F70F96
:100B90001CA383A7018181C72AC682973245EF1023
:100BA000403041016FF03F8203C5418182809378DC
:100BB00008044111639E080095689388482C93733C
:100BC0000801638B03001378E8FF930E000219A855
:100BD000956893880822E5B713731800930E0003F5
:100BE000E30503FE13732800630E03066358060231
:100BF0003306C0409302D0020A8E814F294F63957D
:100C0000E6073373D6023356D602469303430300F6
:100C1000850F050EA30F6EFE7DF20DA01373480025
:100C20009302B0026317030093728800B33250003E
:100C3000960279F2930600035480854FFE8663D3B3
:100C4000FF00BE8613781801158F631308046385AF
:100C500002006353E0007D172A86B308E500130302
:100C6000000221A88142F1B71373F600118271BF0F
:100C70006374B6002300660005063388C840E34964
:100C800000FF3A866353070001467D173295118FA6
:100C9000638802006374B500230055007D170505C5
:100CA00063870302AA96130800031DA86374B600A5
:100CB0002300D60105063388C840E34900FF3A8681
:100CC0006353070001467D173295118FE1BF2A86D5
:100CD000B308E500CDB76374B50023000501050531
:100CE0003386A640E3C9CFFEFD56FD1F6383DF00B8
:100CF00099E7AA873306E5001308000231A8637656
:100D0000B5003306F101102210A10505F9BF63F407
:100D1000B700238007018507B306F640E349D0FEFC
:100D20006353070001473A9541018280EFF26FE774
:100D30002A849D3D09C523AC81806FF0CFE8EF0088
:100D4000F05775D900D9D5BF0D47AA876376C7007C
:100D50009377350091C7AA873E966397C70682802E
:100D600093F7F50F13978700D98F139707015D8FBE
:100D7000B308C500AA87BD463388F84063EB060375
:100D800093574600C156B386D7029207AA970D48DB
:100D900036963383C700BE86B308D3406362180318
:100DA00013572600F156B306D7020A07BA973696AC
:100DB00065B798C3D8C398C7C10723AEE7FE6DBF18
:100DC000910623AEE6FEC9BF8507A38FB7FE71B7B4
:100DD0003D47AA876377C700B367B5008D8BA5CB66
:100DE000AA8701476315C708828003A80700C107C7
:100DF0004107232807FF03A847FF232A07FF03A86B
:100E000087FF232C07FF03A8C7FF232E07FF338884
:100E1000F840E3EC06FD9356460013974600B307EF
:100E2000E500BA954157B386E602014736968D46EE
:100E30003308E64063C306031357260093162700C2
:100E4000B697B695F1563307D7023A9659BFAE8793
:100E50002A87B388C500BD465DBF3388E500832877
:100E600008003388E700110723201801D1B7B386A3
:100E7000E50003880600B386E70005072380060126
:100E800095B763F2A504B386C500637ED50293458A
:100E9000F6FF8147FD176393F50082803387F600E4
:100EA000030807003387C7002A9723000701DDB72F
:100EB0003387F500830607003307F500850714A381
:100EC000E318F6FE82808147E5BF0DC6AA87850537
:100ED0000387F5FF85079306F6FFA38FE7FE09EB6F
:100EE0003E9685076393C7008280A38F07FED5BF18
:100EF0003686F1FE828001476314E600814739A8F7
:100F0000B307E50083860700B387E5009C23B3871A
:100F1000F640E207E18799E30507F9FE3E85828006
:100F2000AA870387070001E73385A74082808507EA
:100F3000CDBFEFF28FC42E89B30B250141112A8C4E
:100F4000B68563F5AB001349F5FFFD5BC169375A00
:100F500000006284930AB002130B0002FD19130A09
:100F6000CA2B31A8130750026389E7026373740127
:100F70001CA013051400B284138614002A8483076E
:100F80000600EDF363060900637C742F2300040060
:100F90003305844141016FF0CFC101481307D002EE
:100FA000930630021305000331A0639E57011368B6
:100FB000480026868307160093041600E397E7FE91
:100FC00013680801FDB76395670113688800D5B7FA
:100FD0006395D70013680802E9BF6395A7001368FB
:100FE0001800C1BF138707FDA54663E6E604014765
:100FF000A546294539A03307A70285043E97130764
:1010000007FD83870400138607FDE3F6C6FE03860B
:1010100004009306E002FD57631FD6048387140083
:10102000254693861400138507FD6365A60A81474C
:10103000254529433DA09306A0027D57E399D7FC9F
:101040009841930426009105E35307FC3307E040E1
:10105000136808016DBFB38767028506B29793874F
:1010600007FD03860600930806FDE37615FF63D3AC
:1010700007008147B6848386040013068006014575
:1010800093F8B6FF6395C80013F5F60F8504038641
:101090000400930690066303D60663C5C60693064E
:1010A00080056304D61C63C3C6049307500263081B
:1010B000F61A63757401930750021CA0838704001D
:1010C000130514006387071A637375011CB01305B9
:1010D00024005DB51306A0026397C7009C41938668
:1010E0002400910569B7B684814771B7930630062D
:1010F0006303D60893064006E31DD6FA136828005A
:10110000A94699A0930630076304D60C63C5C602AE
:101110009306F0066301D61693060007E31BD6F884
:10112000FD566315D700136818002147938C4500BE
:10113000C14690411DA893065007E303D6FC9308CF
:101140008007C146E31716F71306C006938C4500C7
:10115000E301C5FE13068006E31DC5FC90419375AF
:101160002800639C051033763601DE852285EFF07A
:101170001FA4E68511B51378080163150802BA8724
:101180009306000229A06373740114A00504FD17DF
:10119000E34BF0FE9307F7FF6343E0000547338717
:1011A000E74005079387450063747401944114A0D8
:1011B00013051400229713060002B306A7406344E8
:1011C000D000BE8555BB6373750110A10505F5B749
:1011D00083AC0500138D450063930C00D28C6685AB
:1011E0003EC63AC442C22D3BB247AA8612482247A5
:1011F0006355F00063D3A700BE8613780801631E11
:101200000800BA871306000231A06373740110A0AE
:101210000504BA877D17E3CAF6FE814763C1D7028A
:10122000B68763D3060081473305F4002A97130677
:101230000002B307A74063CFF600EA8535BB33064B
:10124000F40063777601B385FC00838505000CA26A
:101250008507E9B76373750110A10505D9BF6373ED
:10126000740110A01305140001BB13680804C146E3
:10127000E1BDFD1411B3A146C1BD42064186F5B5DD
:10128000A38F0BFE31B303A5C1818280EFF26F9172
:1012900003A9C181EFF0EFAE11CD1384C181AA84FF
:1012A000084019C1EFF06FBD930530042685EFF0BB
:1012B0002FB504C04A856FF00F918280397126CA1C
:1012C0002ED232D436D62A8654109305F0071385D1
:1012D00041B63EDA36C606CE22CC3AD842DC46DEED
:1012E0008939AA8603A5C18109E9138541B6F13779
:1012F000F2406244D244216182802686262D1384E6
:10130000C18193E704043EAD9307F00763F4D7006F
:101310009306F007138641B68145EFF06FBB1C4082
:10132000A6AFF9B7EFF2EF87375500001305452355
:10133000713737550000130505244937375700002A
:1013400037550000130747268D4605468D45130582
:101350000527AD37375500001305052985376FF090
:101360008F8631C595661377F50F9386061209C7E8
:10137000BA96882205058280C167938707F0E98FB6
:1013800081CB21851377F50F3697082325058280B9
:10139000B707FF00E98F81CB41859377F50FB697AB
:1013A0008823450582806181369508216505828004
:1013B00003A741825C41BA976305F502B62395E223
:1013C00083A60182638FF600938681829042631325
:1013D000F60088C2D44354C1DC43B306E540BA9753
:1013E00094C71045B307C700630FF500B62381EE1D
:1013F000938681828C426393A5009CC25441D4C3DE
:101400005C413E9710C78280EFE2BFF983A501835C
:10141000375500001305852D553583A5C1833755F4
:1014200000001305C52E593D83A5C1823755000024
:101430001305053061356FE01FF9EFE29FF613F7F2
:10144000C5FFE1462E8663F1E60693073500F19B62
:10145000930687FE63EAF6041D8F130687FE23A812
:10146000C1828966511713844182938606EAD8C3E4
:1014700094C323A407001CC0BA9723A0F182C966B5
:10148000938606EAB755000094C3D8C398C781462F
:10149000054693858539138541BEEFF04FBA184054
:1014A00023A4E1826FE03FF2AA85375500001305BF
:1014B000053A2935C5BFEFE2DFEE39C503A7018341
:1014C0001304350071981389018381446366870E84
:1014D000B1476373F4003144FD55138541BEEFF00D
:1014E0008FB883A7818283A541828328090026853E
:1014F0003386B740B3868840138881826368D600FC
:10150000138541BEEFF02FBE81447DA0B384C5009A
:10151000BA2003AE440061E73307CE40930F47FF84
:1015200063EF8F0A138FC183938EC18213038401EB
:1015300083260F0083A30E001389C1839382C18287
:1015400063EF6F061307C4003297896E3383E5009B
:10155000938E0EEA2322C3012324C3002320D30148
:101560000546D8C0B2A003264300B10863041601A3
:101570002E9618C61387C60022972320E90063F42D
:10158000E30023A0E2000967130707EA9AA0639A21
:10159000970083A601820147B22305EE19C32320D9
:1015A000F800138541BEEFF00FB483A78183B10427
:1015B00081C7A2852685829726856FE0DFE00546F4
:1015C0003697B2A02320EF00E3FFE3FA23A0EE005A
:1015D0005DBFE385D7FCDC430547AE9775BF7286D8
:1015E00031BFEFE21FDC3306B5024111328532C64E
:1015F000D9352A8409C532468145EFF0EFF42285BA
:1016000041016FE05FDC45C5EFE21FD883A741834E
:101610002A8491C3829783A741821389418263669A
:10162000F40883A701826372F408FD55138541BE57
:10163000EFF06FA3835764FF930944FF81CB0357F7
:1016400044FF8967938707EA6301F7023755000073
:101650001305C534A531835644FF035664FF37553F
:101660000000CE851305853691398967938707EA8F
:10167000231AF4FE938781829843231B04FE63F4AC
:10168000E90023A037011387C1831C43832684FF0D
:101690004E85958F83260900B386D940B6971CC323
:1016A000013B138541BEEFF00FA46FE03FD1828074
:1016B000B70700209386070001479387070021465C
:1016C0008C426396A500131547003E95828005075E
:1016D000C106E317C7FE01458280EFE2FFCA2A84F4
:1016E0002E85AE89328AE9372A89A92C83244900BC
:1016F000930749006390F4048D2493E909F82304C7
:1017000034012146D2852285EFF02FFC83A7018486
:1017100099C322858297EF00007803274900930739
:10172000C4005CC358C42322F90004C8EF006077EA
:101730006FE0DFC884407DBFEFE2BFC683A741846E
:101740002A8491C3829723040400EF00C074544498
:1017500018489307C400D8C214C31CC85CC4EF0067
:1017600040746FE05FC6EFE23FC22E89AA898937D5
:10177000AA84484589332A841DCDD0448145EFF0A1
:10178000AFDC214623043401A3040400CA8522856A
:10179000EFF0AFF383A7018499C322858297EF000E
:1017A000806FD8409307C40091045CC358C49CC0A8
:1017B00004C8EF00006F22856FE05FC0EFE27FBEDC
:1017C00083A741842A8491C3829723040400EF00F5
:1017D000806C544418489307C400D8C214C31CC872
:1017E0005CC4EF00006C2285393D6FE0DFBD03056E
:1017F00085007D81828023900186938741C0138775
:101800000708DCC39CC3A107E39DE7FE3D47238A8D
:10181000E18423AC018423A6018693874186DCC33F
:101820009CC38280EFE2FFB703A5C186EFF07FB3D0
:101830007D1593173500138541C03E950841130768
:10184000C5FE210523ACE184EFE09F976FE0BFB7B1
:10185000EFE23FB5EF002064839701862A89B1E764
:1018600003A5C186EFF0FFAF7D15131735009387F1
:1018700041C0BA9784439387818580439385C4FE92
:101880006305B4028CC383A7C185238AA18499C34D
:101890002285829783C741811305C4019385840003
:1018A00093F7F70F81EBEFE07F934A85EF00605FDE
:1018B0006FE07FB1EF00405FCDBFEFE29FAE2A84C3
:1018C000EF00605D8347440393064401C19B93E7A7
:1018D0001700230AF40283475403139737009387B2
:1018E00041C0BA97D84314C318CCD4C35CC89387FB
:1018F000C1869443185C558F98C3EF00805A6FE0FF
:101900009FACEFE21FAA2A847923184C544893070E
:101910004401D8C214C35CC81CCC8347540313973A
:101920003700938741C0BA979843631AF70013872B
:10193000C1861C5C144393C7F7FFF58F1CC3952326
:101940006FE07FA8EFE2FFA5B923938701869A2372
:1019500005079AA3B9236FE01FA7EFE29FA4252BE9
:10196000138701861E23FD17C207C1871EA3634B81
:10197000F00023100700352383A7818591C3C93D5B
:101980006FE07FA4392BEDBFEFE2BFA103A48185F7
:101990001923AA842285B5379147230AF402130537
:1019A000C404112E2285A1358547631CF5003C5CDB
:1019B00089EB2285EFF05FD82685E521513D6FE068
:1019C0009FA083A641861307440123A2E186D8C2C3
:1019D0009387418654C81CCCC5B7EFE29F9C2A84EC
:1019E0005105411108CC48C80CD050D014D43A86C7
:1019F00058D49305300236853EC642C4EFF0CFB4CA
:101A0000585410544C5008507117B72600003A969D
:101A1000938686983D21B24722483726000048CC5D
:101A2000230BF402A30AF402232C0402814723228D
:101A300004052324040523280402230A0402232C7A
:101A40000406232E04060147A286130686A6A28555
:101A50001305C404252483A7018799C3228582978F
:101A6000014541016FE03F96EFE2BF935049144DAD
:101A7000795718D954C21307450190C218CD58C9D7
:101A80002D3DEFF0FFDC6FE01F94EFE29F914111DD
:101A9000B2842E8685452A84368946C03AC63EC41D
:101AA00042C2EFF09FC3024892472247B2464A869D
:101AB000A68522851D3741016FE0FF9003A5818532
:101AC0008280EFE27F8C41112E89AA85054532C6BE
:101AD000B684BA893E8AEFF01FC92A8411C92685C7
:101AE000EFF07F9D324609E92285EFF03FCD0144BA
:101AF000228541016FE09F8CAA865288CE87268777
:101B0000CA852285D93DEDB7EFE2BF89692683A753
:101B100081850546AA8603C747033D8B631CC70220
:101B2000D04B984F6308E60258C210C303C6570350
:101B3000938647010E06138741C094CF32975043D6
:101B400014C290CF54C3D8CBA92EEFF07FD001455B
:101B50006FE07F873685B126DDBF834745030547A4
:101B6000BD8B639FE702EFE2DF832A842D26834744
:101B70004403AA842285C19B93E72700230AF40229
:101B8000EFF03FD81305C404F1222685192E83A750
:101B90008187014581C72285829701456FE0BF8219
:101BA0007D558280EFE2EFFF41112AC6ED2403A4A8
:101BB00081852A89228555379304C40470008145A4
:101BC0002685D122268539224A85E12CEFF05FC88F
:101BD0001858F9576314F7002328040201454101FE
:101BE0006FE06FFEEFE2EFFBEFE01F8C653F6FE011
:101BF0008FFD834745030947BD8B6390E704EFE200
:101C00004FFA2A84492C5448184C93074401AA845B
:101C1000D8C214C31CCC5CC81305C404252A26856D
:101C200049242285EFF07FC983A74187014581C7F9
:101C30002285829701456FE00FF97D558280EFE2A2
:101C40004FF68346650305473317D70018DD09476C
:101C5000A30AD502230AE502693F83A7818599C3B8
:101C6000EFF01FBF01456FE00FF65449184D930781
:101C70004501D8C214C31CCD5CC98280EFE26FF26B
:101C80004111B2842E86A9452A8436C63AC43EC282
:101C9000EFF0BFA49247B2462247F99B1CB49307CA
:101CA000440144CC14D02324040258D01CCC5CC87A
:101CB00041016FE04FF1EFE2CFEE2A84E92AAA84D6
:101CC000228565372685F12A2285EFF0FFA601459A
:101CD0006FE06FEFEFE2EFEC2A84752AAA84228589
:101CE00069371C342685F99B1CB4652A83A7C184F7
:101CF00099C322858297EFE04FF85C503E9508D457
:101D0000592A138781880328470037060080938764
:101D100081881346E6FF98436315F8029386C187CE
:101D20009042050690C29306440154C358C894C318
:101D30001CCC1C3493E717001CB4A52201456FE0AE
:101D40008FE8544B0C546385B6008D8EE378D6FC37
:101D5000BA87D1B71C35858B8DC7EFE28FE483A797
:101D600081842A8491C382973D22AA842285EFF040
:101D7000DFEF26853D221C340145F99B1CB46FE042
:101D80008FE47D55828085476381F50263C5B70086
:101D900085C1014582808947638FF5008D47E39AAD
:101DA000F5FE1C3593E7270009A85C511CC2D5B786
:101DB0001C425CD1F9BF1C35F59B1CB5D9BFEFE2C5
:101DC000CFDBEFE08FEB2A8CF920B70900802A8A5D
:101DD0009384818893C9E9FF8D4B804063169400FA
:101DE0005285C1206FE0EFDC48481309C4FE33057B
:101DF000AC40E3E7A9FE83A7018899C34A8582978F
:101E00004A85EFF09FE61C4448448297EFE0EFE6F6
:101E100083A741882A8C99C34A858297834754FFB8
:101E200013F7E70FA30AE4FE8D8BE39877FB4A854F
:101E3000EFF05FEA5DB793878188DCC39CC3828043
:101E400082801106719A2A8837C7ADDE130506F81D
:101E5000AA871307F7EE631EF600A167938707882A
:101E60002322D6F82324B6FA232006F92324F6F8F1
:101E7000828098C39107C5B737F700E01C43B706C7
:101E80000080D58F1CC3828037F700E01C43860793
:101E900085831CC382802165130505807315053079
:101EA0008280731005308280EFE2AFCF1387818983
:101EB00018439387818919E323A8A18823AAB188AD
:101EC000054798C3553F6FE00FD02A8781471843D5
:101ED0006314A7003E8582808507D5BFB707EFBE94
:101EE00037E700E0938707083CC701458280EFE2AF
:101EF0004FCB375500001305C53DEFF02FBC014512
:101F00006FE06FCCEFE2EFC92A84FD54376900001F
:101F10007D14631494006FE00FCB130549B4EFF008
:101F2000EFB9FDB7EFE24FC60041AA843769000060
:101F3000B7690000631494006FE04FC89305C4FEB6
:101F4000130589B4EFF08FB71C40638697001385A3
:101F5000C9B4EFF0AFB60040F1BFEFE28FC42E89F5
:101F6000EFE01FFC2A84EFF0FF9D83240900639CAF
:101F70002401EFF09F9EA14763C3870011E0214435
:101F800022856FE04FC4138544FFEFE07FF9635370
:101F9000A4002A848440E1BFEFE22FBE0545EFF0A4
:101FA0002FF1B7590000130945002A84CA8513850B
:101FB0000969EFF09FFAAA85AA84375500001386B5
:101FC000096913058569EFF06FAF2685EFF09FF380
:101FD000375500001305C56DEFF04FAE4040B759BF
:101FE0000000054A894A375B0000B75B0000375C98
:101FF0000000B75C0000375D0000631589000145F3
:102000006FE02FBB034794021385C971930644FF09
:102010002146A685EFF08FAA8347840213858C7230
:10202000BD8B638E470113054C73638A570113857B
:102030000B7491C711476396E7001305CB74EFF05B
:10204000EFA74C4C93073002AE8698226306F70246
:102050001050930740060848B295B386D540B38622
:10206000F602585C5C50898D13058D75B3D6C60297
:10207000EFF0CFA4004051B78506C1BFEFE2CFB06B
:1020800041110945EFF0CFE29309450037590000AF
:102090002A84CE8513050963EFF03FECAA85AA8454
:1020A00037550000130609631305C563EFF00FA150
:1020B0002685EFF03FE53755000013058565EFF005
:1020C000EF9F4040375A0000B75A0000376B0000BE
:1020D00063968900014541016FE04FAE1A281C4408
:1020E000930644FF1309840036C63AC44A85630642
:1020F000F902EFF09FDD2247B246AA872146A68566
:1021000013850A67EFF08F9B4A85EFF0BFE1130557
:102110008B60EFF0AF9A004065BFEFF01FDB224706
:10212000B246AA872146A68513050A68EFF00F99E3
:10213000DDB7EFE26FA541111145EFF06FD79309BD
:102140004500375900002A84CE8513054947EFF032
:10215000DFE0AA85AA843755000013064947130516
:10216000C547EFF0AF952685EFF0DFD93755000072
:102170001305054AEFF08F944040375A0000B75AD4
:102180000000376B000063968900014541016FE054
:10219000EFA21C4413098400930644FF1848630906
:1021A000F9024A8536C63AC4EFF03FD22247B2461A
:1021B000AA872146A68513850A4CEFF02F904A8501
:1021C000EFF05FD613058B60EFF04F8F004065BFD7
:1021D0002146A68513058A4DEFF04F8EC5BFEFE26D
:1021E000AF9A41110D45EFF0AFCCB759000013097C
:1021F00045002A84CA851385C95CEFF01FD6AA85DD
:10220000AA84375500001386C95C1305455DEFF0BD
:10221000EF8A2685EFF01FCF375500001305855F45
:10222000EFF0CF894040B75900006316890001459F
:1022300041016FE0AF98930644FF1305840036C652
:10224000EFF0BFC8034834015C48B246AA88214772
:102250002146A68513858961EFF04F860040F1B7CE
:10226000EFE28F9241111545EFF08FC493094500BD
:10227000375900002A84CE851305C94EEFF0FFCDF3
:10228000AA85AA84375500001306C94E1305454F89
:10229000EFF0CF822685EFF0FFC63755000013051B
:1022A0008551EFF0AF814040375A0000B75A000027
:1022B000376B000063968900014541016FE00F9084
:1022C0007A285E281044930644FF1309840036C61A
:1022D0003AC43EC24A856307C902EFF01FBF924766
:1022E0002247B2462A882146A68513854A53EFE045
:1022F000FFFC4A85EFF01FC313058B60EFE01FFC66
:1023000000404DBFEFF07FBC92472247B2462A887B
:102310002146A6851305CA54EFE05FFAD5B7EFE270
:10232000AF8641111945EFF0AFB893094500375911
:1023300000002A84CE8513054956EFF01FC2AA85F6
:10234000AA84375500001306495613050557EFE0D8
:10235000FFF62685EFF01FBB375500001305C55863
:10236000EFE0DFF54040375A0000B75A0000376B06
:10237000000063968900014541016FE02F841A2C0B
:102380001C44930644FF1309840036C63AC44A85A8
:102390006306F902EFF07FB32247B246AA872146CF
:1023A000A68513854A5AEFE07FF14A85EFF09FB783
:1023B00013058B60EFE09FF0004065BFEFF0FFB0CA
:1023C0002247B246AA872146A68513058A5BEFE01D
:1023D000FFEEDDB7EFD25FFB5D712545EFF04FAD4E
:1023E0009565130600052A84130945009385850821
:1023F0000A85EF20B037B7590000CA851385C94058
:10240000EFF0BFB5AA85AA84375500001386C940EE
:1024100013054541EFE09FEA2685EFF0BFAE375543
:1024200000001305C543EFE07FE94040D149375A2A
:10243000000063168900014561616FD03FF81C44BC
:10244000930644FF63E0F90298088A07BA9703A746
:1024500007FB1C282146A68513050A46EFE01FE668
:102460000040C1BF4647F5B7EFD21FF22945EFF054
:102470002FA4B7590000130945002A84CA85138583
:102480000978EFF09FADAA85AA843755000013861E
:10249000097813058578EFE07FE22685EFF09FA6A7
:1024A000375500001305057BEFE05FE14040B75969
:1024B0000000375A0000B75A0000631E8900EFD0B1
:1024C000DFFBAA853765000013058580EFE01FDF7D
:1024D00001456FD0BFEE5C4C184C1385497D9306C7
:1024E00044FF2146A685EFE07FDD8347D4FF1385B7
:1024F000CA7E858B99E313058A7FEFE03FDC0040BD
:102500006DBFEFD27FE8375500001305453EEFE081
:10251000FFDA03A4018AB7590000375A000083A7E5
:10252000418A6365F40001456FD05FE904400946C4
:102530009385893F2685EF20903219C55040A685A6
:102540001305CA3FEFE09FD73104D1BFEFD2DFE3DD
:1025500037650000130585CAEFE05FD603A4018A42
:10256000B7690000376A000083A7418A636BF400F3
:102570003765000013058560EFE05FD401456FD03B
:10258000FFE304401946938549CC2685EF20302D82
:1025900001E95040938564001305CACCEFE01FD2D7
:1025A0003104D9B705458280EFD21FDE79712A84C4
:1025B000AA9593060002254783070400B38485404B
:1025C0006385D70A6383E70A0145638B04100149D9
:1025D00013070002A546B307240183870700638A17
:1025E000E7086388D7086314990883A9018A83AA36
:1025F000418A376B000063F0590903AA09001946A4
:1026000093054BCC5285EF20902559E54A86A2854B
:1026100013056A00EF20B02441E14A9A83076A005B
:10262000A5EF83A989006388090413068002814508
:102630002800EFD01FDA13098100CA86A28701455E
:10264000014713080002A548294313062002130E70
:10265000C005838507006384050163961505631F24
:102660009702A9476303F50469A80504B1B70509F2
:102670009DB7E31C09F6A287038707001377F7FDD0
:1026800079E737650000130505C923800700A28597
:10269000EFE0DFC27D55A9A0B109B1BF23800700DB
:1026A000050785077DB763106504376500001305CE
:1026B000C5C6EFE0BFC00018B7640000832509005D
:1026C0001385C4C81109EFE07FBFE31989FE3765A0
:1026D000000013058560EFE07FBE29452C0082993C
:1026E00045616FD0BFCD637E970005056392C50439
:1026F000850705079CC2838507006381C502636463
:10270000970069FD8DBF838E17006396C5016394A2
:10271000CE008507050785070507F1BFE37397FE20
:1027200023800700050785079106E36497F2D1BF70
:102730009CC2838507006389050163871501E30255
:1027400097FC85070507F5B7E36097FE5DBF850732
:1027500025B7EFD29FC28307050099E78145014560
:10276000EFF0DFDE6FD0FFC403AA018AAA8981449B
:102770000149376B0000B76B000083A7418A63698A
:10278000FA00EDD04A86A6854E85EFE00FF4D9BF5A
:1027900003240A00194693054BCC2285EF20300C08
:1027A00021E14E85EF20900A19042A86A2854E85E4
:1027B000EF20F00A15E5631709002285EF201009C4
:1027C0002A89A284A68722870386070001EE858FC7
:1027D00063D327013E89A28513854BCDEFE01FAE61
:1027E000310A61BF83060700FDD2E312D6FE8507DA
:1027F0000507D9BFEFD2FFBAEFF00FFA01456FD04E
:102800009FBCEFD21FBAEFE03FC001456FD0BFBB06
:10281000EFD23FB903A5C189EFE0EF8C01456FD03E
:102820009FBAEFD21FB8B76700009387476123A014
:10283000F18AB76700009387477623A2F18AB767CA
:1028400000009387477623A4F18AB7670000938737
:10285000477693050021054523A6F18A1384C18993
:10286000EFE03FD808C019E937650000130585D8A7
:10287000EFE0DFA47D5422856FD0FFB4B7350000B0
:1028800037650000A9472D47930600400146938510
:10289000259A130505DAEFF0CFA2AA840840B765A0
:1028A000000081460146938585DAEFD05FF9014447
:1028B000F9D02685EFF0AFB87DBFEFD29FAEEFF035
:1028C0007FCE0DC5B7650000938545D5138541C8FA
:1028D000EF20C076B7650000938545D6138541C8C3
:1028E000EF20E073138541C86FD0FFADB7650000DE
:1028F0009385C5D5E1BFEFD2DFAA2A8437650000F2
:10290000130545DCEFE09F9BEFF03FFBAA853765A1
:1029100000001306A41B1305C5DCEFE03F9A014538
:102920006FD07FAAEFD2FFA741112AC6EFD07FC593
:10293000B24511E937650000130585D6EFE01F9811
:1029400041016FD05FA883A7C189AA841384C1897C
:1029500083A7C720E386A7FE93053014EFD05FCA94
:1029600065F11C4003A5C72009C9EFD01FD11C4049
:10297000814503A5C720EFD09FD70040130600056F
:1029800081451305A41BEFD0DFA4B7350000231544
:10299000042023269420938505812685EFD03FD5FA
:1029A00045B7EFD21F9D83A7C18941119384C18987
:1029B00003C74702136717002382E70283A7C720D4
:1029C00091E7EFE05F8C19C1EFF0DFF5EFF0FFEE7C
:1029D000EFE0DF8E376B0000B76B0000B7690000D7
:1029E000376A0000B76A0000376C0000B76C00005F
:1029F0009C4085461306F10003A5C720FD55EFD086
:102A00005FCB8547631AF5000309F100ED4780406D
:102A10006319F90008D0E9BF8840FD55EFD0BFE445
:102A2000C1BF1C506392A7029307B0056315F9005C
:102A300089471CD075BF23200402E30B09FAA54780
:102A40006314F9120149D1A80947E398E7FE23204E
:102A50000402930710046312F9046E30D1D9FD15F6
:102A6000C205C1816EB09307A41B13070005B3858F
:102A7000E502130600053E859385A502A295EF2089
:102A8000E04EEF20A05C1375F50F2305A420A305ED
:102A9000A4202285EFF03FE6A1BF93072004631135
:102AA000F90216347E301387F6FF63D8E7008507F6
:102AB0007EB09307A41B6E304DBF9DDA7AB0D5BFB0
:102AC000930740046310F9028347B42095D313851C
:102AD00009DBEFE0AFFE98408347B720FD17A30561
:102AE000F72039B793073004E319F9F48347B4208A
:102AF0000347A420E3FEE7EE3E948305A41B138561
:102B00004ADBEFE0AFFB98408347B7208507C1BFA2
:102B1000138509DBEFE08FFA050980408347B42075
:102B2000E348F9FE13058A60EFE04FF9EFF09FA745
:102B300085471304A41B6315F5002285EFF07FC1C0
:102B4000EFF0BFD72286AA851385CCDCEFE00FF724
:102B500080401305A41BEF20604F1375F50F23056C
:102B6000A420A305A42069B59307F0076305F90025
:102B7000A1476315F9088347B420E38B07E60346B2
:102B8000A420FD1793F7F70F7D161376F60F230594
:102B9000C420A305F42063F8C7049385B71B1385ED
:102BA000A71B1D8EA2952295EFE0AFAD9C4013852B
:102BB0008BDB03C7A7203E97230D071A83C5B720D9
:102BC0009385A51BBE95EFE06FEF9C4003C4B72033
:102BD0009C4083C7A720E3CD87E0138509DBEFE0A6
:102BE000EFED0504F5B713050BDCEFE02FED9C408E
:102BF00003C7A720BA97238D071ADDBB3547834744
:102C0000A4206305E9002947631EE90EB9CB0359E7
:102C100084029147130DA41B63FB2709930DA4168F
:102C200013060005EA856E85EF2000321DC91309E1
:102C3000A4024A851309090513060005CA85EF2079
:102C4000E032E3982DFF1306000581456E85EFD035
:102C50004FF80346A420EA856E85EF202031954782
:102C60001EB41E347EB0EFF0FF9385476312F50269
:102C70009C4083C74702858B89C713058A60EFE0B4
:102C8000EFE388408345A5201305A51BEFF0DF91F6
:102C9000EFF0BFC2EFE08FE28040130600058145F0
:102CA0001305A41BEFD0EFF22315042091B36301A9
:102CB00009021305F9FF930700053305F502130612
:102CC0000005EA851305A5022295EF20E02751D9DA
:102CD000930D00053305B90313060005814513055F
:102CE000A5022295EFD0EFEE0A340346A420EA8530
:102CF0003305B5031305A5022295EF2020271E34C6
:102D00008507B9BF1307F0046374F7002305042097
:102D10000346B4208347A4206370F6089305A61BDE
:102D20001305B61BA2953386C7402295EFE06F9539
:102D30008C4083C7B5203387F500230D271B03C7BD
:102D40004502058B01CB9387A71BBE9513058CB459
:102D5000EFE0CFD69C4003C4B7209C4083C7A72098
:102D60006346F40298408347A7208346B72085072F
:102D7000850693F7F70FA305D7202305F7209306C1
:102D8000F004E3F7F6C6231507209DB1138509DB90
:102D9000EFE0CFD20504D1B7A297238D271B83473D
:102DA0004402858BE1D3CA8513854ADBEFE00FD15E
:102DB00055BF7C4123280504232A05049C4381CB6D
:102DC000EFD22FDE9305850482976FD0CFDF0145C8
:102DD0008280EFD26FDB36899DCAAA843284B30920
:102DE000D600294A1C20639B4701BE2C93F7070499
:102DF00091C7FC40B54526859C478297FC408305DA
:102E0000040026859C4705048297E31D34FD4A850E
:102E10006FD0CFDAEFD2EFD893F705102A8491C79D
:102E20001A2D61551377071035CF13F7054011C7D9
:102E30001A2C61551377074035C713F7050493041F
:102E4000000401E7262C93F40404384893F5F50FA9
:102E50002EAC39EBA1C76844298142054181310577
:102E6000EFE06FE570442A893105298242064182EC
:102E700081452320A900EFD03FED232209003E2CFD
:102E8000232409002328240593E707103EAC7C4047
:102E900013060010C145DC43228582973E2C014574
:102EA000DD8C26AC6FD02FD2F5DB93E505102EAC70
:102EB000F5B70948AA8763810503EFD28FCE0D4885
:102EC0006382050305476399E5041A2D1377F7FD1F
:102ED0001AAD01456FD02FCF1A2D136707021AAD17
:102EE00001458280328775D6504274454C2D298227
:102EF000A9824206C2064182C1826304D6001D45F2
:102F0000F1F91443B4C75443F4C7E1D5F443BA8587
:102F10003E859442829675BF7C41DC4382975DBFBB
:102F2000EFD28FC63684B1CA3E2DAA89328993F773
:102F30000710B6849DE37D5AA94A83A749044E85AC
:102F4000DC478297630945012300A900FD140509A8
:102F500063035501FDF0058C0DA02449368A854A8E
:102F6000EFE07FF3FE20DA202A869444631AF7000C
:102F700081EAEFE01FF33304444122856FD00FC490
:102F800098403E97034B070003A7C9048507C20773
:102F90002983C1834207FEA0418363E4E7002393B2
:102FA00004006394560123A404003285EFE07FEF10
:102FB0007D1A230069010509E3140AFA6DBF582D33
:102FC000854763ECE7023E2D93F707109DC7EFD2CC
:102FD0004FBD2A842849EFE00FE33E2C2328040448
:102FE0001306001093F7F7EF3EAC7C40C5452285F1
:102FF000DC43829701456FD00FBD01458280EFD23F
:103000004FBA37370000130727DB18D537370000D2
:10301000130747E158D5373700001307E7FB18D9E6
:1030200037370000130707F258D937370000130766
:1030300027DD18DD37370000130727EB420658DD80
:1030400034C14182232A05002320050223220502E0
:10305000EFD0CFD76FD02FB793F5F50F854763919A
:10306000F50AEFD26FB220494111AA847D598549F2
:10307000FC402685DC4782972A8A63072505EFE016
:103080009FE15A201C40BA97238047015E20F844F4
:103090008507C2072983C18342075EA0418363E499
:1030A000E7002312040076205E20639CD70085078A
:1030B000C207C1837EA02324340163E4E700231305
:1030C0000400EFE01FDE6DB79C5085C3EFE0BFDC6E
:1030D0005A206E20636EB700B305B7402EC6EFE0EE
:1030E0005FDC9C50B2452685829741016FD00FADC1
:1030F000FC44998DA983C207C183B385B740F9BF4A
:10310000828001CEEFD2EFA97841B2878E23184397
:103110003222029701456FD00FAB7D558280EFD2EE
:103120004FA8138781D078432E86AA85184313852C
:1031300081D002976FD02FA9EFD2AFA6138781D08D
:1031400078432E86AA855843138581D002976FD085
:103150008FA7EFD20FA5138781D07843AA85138557
:1031600081D0184702976FD00FA605C6114763920A
:10317000E602EFD20FA37C410E2241119C4736C6D6
:1031800032C482972246B2462AA2368541016FD0C8
:103190008FA38146368582801DC2B2871146639017
:1031A000C602EFD20FA07841B2238E2358434111BB
:1031B00036C60297B246410136856FD0CFA0814610
:1031C00036858280EFD2EF9D938781D04947D8CB57
:1031D000373700001307A716D8DB3737000013076F
:1031E000871998DF3737000013072710ECC3B0C3E7
:1031F000AA850D46138581D023A0070223A20702CA
:1032000023A4070223A6070223A80702D8DFEFD0D2
:10321000EFBB01456FD02F9B370500201305857943
:10322000828037150020130585798280EFD26F9751
:10323000B707002003A787249307803EC156335762
:10324000F702B7E700E02386D7402387D74085669B
:1032500023A0D710916623A0D710B7F700E023A0D2
:10326000070023A20700014690C78146D4C78146C4
:103270001306F7FF90CBD4CB3D4798C3EFD04FA6B2
:10328000EFF09FF92A84EFF0DFF9AA852285EFE0BD
:10329000CF9A37650000130545E4EFD03FFF6FD0AC
:1032A0008F9273110134EFD07F8AB7F700E023A229
:1032B0000700EFD0EF9CEFD05F8C731101347300E7
:1032C0002030232605000CC150C1232405000545EC
:1032D00082805C45544118458507B3E7D702638E69
:1032E000E70058451C41BA978CA35C4558418507B7
:1032F000B3E7E7025CC505458280795582801845B1
:103300005C45630FF70018451C41BA979C239CA1AC
:103310001C4558418507B3E7E7021CC50545828077
:10332000014582805C4518454841998FAA9733E54D
:10333000A702828081478546130700023396F60074
:103340006306A6008507E39BE7FEFD573E85828066
:10335000EFD22F85854513050002EF10405F6FD037
:103360008F86EFD20F8485452145EF10405E6FD0E8
:103370008F85EFD20F8385451145EF10405D6FD0EB
:103380008F84EFD20F8285454145EF10405C6FD0AE
:103390008F83EFD20F81854513050004EF10205B6A
:1033A0006FD06F82EFC2FFFF99653765000001465D
:1033B0009385C5E413054553EFF0DFE06FD0AF8090
:1033C0009307400663ECA7009317450019651305A2
:1033D00045EE3E951841FD576313F7000145828085
:1033E000EFC23FFC411113F5F50F32C6EFF05FFD60
:1033F00011C54E2532460845EF10C03541016FC05A
:103400009FFCEFC21FFA13F5F50FEFF07FFBAA87C1
:10341000014589C7CE278847EF1020336FC0BFFA18
:10342000EFC23FF8011113F5F50F3284EFF05FF9A9
:1034300005C55C412AC6829732455C45FC82C1477E
:103440003ECE8D473ECC09C41547631AE40002CE38
:1034500008454C08EF10602305616FC0DFF6054793
:103460006315E40091473ECEE5B76315F40093077A
:103470008002D5BF89476315F40093078004E5B740
:1034800091476314F400D147F9BF99476314F400DE
:10349000F147D1BF9D47E31DF4FAE147E9B7EFC219
:1034A000BFEE13F5F50FAE84B289368A3A89EFF094
:1034B0003FF1994731CD4845EFF0DFE73D472A849A
:1034C00099476367A704EFE01F9DB146B306D40296
:1034D000B7070020138707082A86938707083697BF
:1034E00083160700639F96004C43639C45012E237F
:1034F00063993501184763162701EFE09F9A8147CA
:1035000001A87D576389E6003285EFE09F999D47CA
:103510003E856FC0BFEA31453305A4023E9506A142
:103520002322450123113501232425013285F1B7DA
:10353000EFC23FE713F5F50FEFF09FE819471DC9FC
:103540004845EFF03FDFBD472A84194763E4A702EF
:10355000EFE07F94B1473304F402B707002093876C
:1035600007087D57A297839607006398E600EFE06F
:103570005F9301473A856FC01FE541677D1798C388
:1035800023A2070023A40700DDB7EFC2FFDF01116C
:1035900013F5F50F328AEFF0BFE2994721C1854458
:1035A0002A8463159A104845EFF0DFD83D47AA8476
:1035B00099476365A702EFE01F8EB14AB3875403B2
:1035C0003709002013090908AA893E990317090041
:1035D000FD576319F700EFE0DF8C99473E850561E1
:1035E0006FC0DFDD5C40829785450545EF102036D2
:1035F0005C440D473AC47C823EC88357290002CA06
:1036000052CE638C4709C1C70947638DE708084458
:103610004C00EF1080071844B7170140938607C08D
:1036200005456302D7020945630FF70093870740FA
:103630000D45630AF700B7270140938707800145CE
:103640006313F700114593F5F40FEF1040110808CC
:10365000EF00907A9967938747E68E04BE94D04036
:1036600037E700E093060005B307C7002380D74083
:10367000935756009387070485468A07B396C6007A
:10368000BA9794C34E85EFE0DF81814781BF9307EE
:1036900080023EC6A1473ECC9DBF930780043EC634
:1036A00056CCB5B791473EC6C147F5B79947E31722
:1036B0000AF24845EFF01FC83D479947E360A7F27B
:1036C000931735001965130545E63E955841935704
:1036D000570093870706B394E4008A0737E700E0B2
:1036E000BA9784C35DB7EFC2DFCBEFF0BFC4B14779
:1036F0003305F502B7070020938707083E955C4124
:1037000099C3084582976FC01FCC73110134EFD065
:10371000EFC30545EF00F07419C50545EFF0BFFC98
:103720000545EF00F075EFD04FC5731101347300FC
:10373000203073110134EFD06FC10945EF00707272
:1037400019C50945EFF03FFA0945EF007073EFD056
:10375000CFC2731101347300203073110134EFD0E4
:10376000EFBE1145EF00F06F19C51145EFF0BFF73F
:103770001145EF00F070EFD04FC0731101347300AA
:10378000203073110134EFD06FBC2145EF00706D14
:1037900019C52145EFF03FF52145EF00706EEFD0E0
:1037A000CFBD731101347300203073110134EFD099
:1037B000EFB94145EF00F06A19C54145EFF0BFF29E
:1037C0004145EF00F06BEFD04FBB73110134730034
:1037D000203073110134EFD06FB713050002EF00F2
:1037E00050681DCD13050002EFF0FFEF1305000434
:1037F000EFF07FEF13050008EFF0FFEE1305001068
:10380000EFF07FEE13050020EFF0FFED1305003E13
:10381000EF001067EFD06FB67311013473002030E2
:1038200013050004EF00F06355FD13050008EF00D9
:1038300050634DF913050010EF00B06245F5130514
:103840000020EF00106259FDF1B773110134EFD081
:10385000EFAF13050040EF00D06029C11305004011
:10386000EFF07FE8056513050580EFF0DFE70565FC
:10387000EFF07FE70965EFF01FE71165EFF0BFE6B6
:103880002165EFF05FE64165130505C0EF00505F6D
:10389000EFD0AFAE7311013473002030056513050E
:1038A0000580EF00105C5DF90565EF00905B5DF54C
:1038B0000965EF00105B5DF11165EF00905A59FD4D
:1038C0002165EF00105A59F9E1B701458280EFC236
:1038D0005FAD9C412041A14641111CC0B1473EA4AF
:1038E000DC412316040013F7F7006301D702A54655
:1038F000631ED70005675AA013D747000D8B01C779
:1039000085466308D7002313040031A02312040066
:10391000E5B709677AA099838D8B05476389E7002E
:1039200081C709476389E7062314040021A0930790
:1039300000601EA41848B7470140938707806318AA
:10394000F704116585451105EF106000930700200D
:10395000B71401407C820D49E1474C001385048077
:103960003EC64AC4EF007052930700407C824C0070
:103970009147138504803EC64AC4EF0010510848A1
:10398000A285EF10800008488545EF100009014529
:1039900041016FC05FA39307004061BFEFC2DF9E8C
:1039A000B71400201384047F930750035CC83719B1
:1039B0000020B74701401306897993870780744632
:1039C0001CC89967938787537CC2B70700C0F58FDF
:1039D000C166A106716713070720D58F11654111D4
:1039E00038C67CC68545B7070C00110518C01CC435
:1039F0002322040023160400EF007075B71901405C
:103A0000930700207C820D4AE1474C001385098012
:103A100052C43EC6EF007047930700407C824C00C2
:103A20009147138509803EC652C4EF0010460848EE
:103A30009385047FEF00707508488545EF00F07DA1
:103A4000B76500009386047F13063010938545E424
:103A500013058979EFF0AFDA014541016FC01F9678
:103A6000EFC23F942041930500020848EF10A000E8
:103A700019C51C48CA231375F50F6FC0DF947D5517
:103A8000EDBFEFC21F9224412E84884893050004A5
:103A9000EF00707E7DD99C4842044180C2A3054559
:103AA0006FC07F92EFC2FF8FC1473841638BF50231
:103AB000C5476395F502544B054693D75600938747
:103AC00007063316D6008A07B7E600E0B69790C31C
:103AD0000146084B93055052EF00907501456FC0A9
:103AE0009F8E544B054693D7560093870704331691
:103AF000D6008A07B7E600E0B69790C30546D1BF67
:103B0000411122C626C473110134B7140020EFD02E
:103B1000EF8393878479A043930550520848EF00C0
:103B2000307619C9854513858479EFF0EFD20848BE
:103B300093055052EF009078EFD02F847311013429
:103B40003244A24441017300203073110134EFC0AC
:103B5000FFFF3765000013058555EFD02FF6EFD036
:103B6000CF81731101347300203073110134EFC021
:103B7000FFFD376500001305C554EFD02FF4EFC0EB
:103B8000DFFF7311013473002030EFC29F8137656E
:103B9000000013058556EFD06FF2B12AB707002059
:103BA00083A58724376500001305C557EFD00FF1B3
:103BB000EF00F023AA85376500001305C558EFD044
:103BC000EFEF2D2001456FC01F80EFC28FFDEF008A
:103BD0003070EF00F0706FC00FFFEFC28FFCEF008E
:103BE000407759253525992D6FC0EFFDEFC26FFB4A
:103BF000EFF0BFFDEFF07FFE6FC0EFFCB7170240A4
:103C00009843B706FFF041111367170098C3D843D4
:103C100037060200758FD8C39843B706F7FEFD1626
:103C2000758F98C39843B706FCFFFD16758F98C330
:103C3000D843B70601FFFD16758FD8C39843B70662
:103C400000ECFD16758F98C33707FF0098C723A6B1
:103C5000070202C402C69843C166558F98C3B716BF
:103C6000024005679C42F18F3EC6A24785073EC4CD
:103C7000B24781E7A247E397E7FEB71702409C43AC
:103C80001397E7006357070685473EC632478547C7
:103C9000631FF704B7170240D843B706C1FFFD16EC
:103CA000D8C3D843D8C3D84313670740D8C3D84331
:103CB000758FD8C3D843B7062900558FD8C398430A
:103CC000B7060001558F98C3984393166700E3DD4C
:103CD00006FED843B7160240719BD8C3D84313677A
:103CE0002700D8C32147DC42B18BE39EE7FE4101A8
:103CF000828002C661BFB7160240D842B7070020D3
:103D00001146318B938787246305C70021466308DA
:103D1000C70237177A001307072098C337170240E6
:103D2000584311839376F7003707002013070714D1
:103D30003697142398433357D70098C38280D842CC
:103D4000D442416649833D8BF18E1306270015CF7F
:103D50003D47630FE6024147630FE6024547814551
:103D60006313E6004146A1E237470240032707807C
:103D7000418B0DC737177A00130707203306C70298
:103D800090C3C9DD9843058349BF81454946E1BFDA
:103D900085453546C9BF81453D46F1B737173D00DA
:103DA00013070790E1BF3715024058559316F700E7
:103DB000585563DF060411833D8B930617003717B0
:103DC0007A00130707203357D70298C35455A182AE
:103DD000BD8A8DE295463307D702058398C337170E
:103DE0000240585794433D8B050733D7E60298C3EA
:103DF000984369B705456394A600E546E9BF3D458C
:103E00006396A600D1463387E602C9BF8906E5BF9F
:103E10003D8B9306170037177A0013070720335797
:103E2000D702F1B701A07390123497D1FF1F93818D
:103E3000E1C117C100201301E11C17350000130573
:103E4000659497C5FF1F9385E51B1386818063FAF0
:103E5000C5008322050023A0550011059105E3EA62
:103E6000C5FE1385818097E5FF1F938525CF637776
:103E7000B500232005001105E36DB5FEFD427390EA
:103E800002BCFD4273904280B782000093820280A0
:103E90007390023097C2FFFF9382021793E23200C1
:103EA00073905230EFF09FD597C2FFFF9382026D5F
:103EB0007390123473002030EFC2AFCE2A893725B9
:103EC00000203284AE845946814513052584EFC015
:103ED0004FD0B72500209387C5830547D8A3C0B32B
:103EE00023AE258381471387C58363E8870203A533
:103EF000018B22869385C583EFC09FAC19C53765BA
:103F000000001305C559EFD06FBB376500001305DE
:103F1000C55AEFD0AFBA6FC00FCBB386F400902272
:103F2000B306F7008507F0A293F7F70F7DBFEFC246
:103F30004FC72A89372500203284AE8461468145E7
:103F400013050584EFC0EFC8B72500209387C5830C
:103F5000C0B323AE258381471387C58363E28702FD
:103F600003A5018B22869385C583EFC07FA519C564
:103F7000376500001305C559EFD04FB46FC0AFC40B
:103F8000B386F4009022B306F7008507F0A293F7FA
:103F9000F70FE9B7C16769768146FD1705061397E4
:103FA000060141836364B7003E8582803307D500F4
:103FB0001823B98F214713F817008583630508007C
:103FC000B18FC207C1837D17420741836DF7850614
:103FD000F9B7EFC26FBB370400208327041598356B
:103FE0002A89AE84B289130404156314F7005C4077
:103FF000829798341C446317F7005C444E86A6856C
:104000004A8582976FC08FBBEFC2AFB64111AA8BB2
:10401000412B61C97945EFD0FFBC5E85D123AA85CC
:10402000376500001305855BEFD04FA9B72A002044
:1040300013062003814513858A8093898A80EFC007
:104040004FB90149014B81440144894C138A8A804C
:10405000130D0003138C19005E85592359C15E8529
:10406000A12B937DF50FB3878900130614002380DD
:10407000B70163049601638E040EB70700208346E0
:104080000A0083C70716639BF600B70700209387D3
:10409000071683461A009C336389F6002286E28560
:1040A0004E85EF00B06C22861DA8A9476304F60078
:1040B00063F49C0C83479A006382A70D9306100A51
:1040C0006383D70AA68763F3940189472286E28532
:1040D0004E8593F4F70FEF0070692286014B6377EA
:1040E000CD0A41016FC0AFACE31B26FF83479A00A6
:1040F0006392A7059305D6FF93F5F50F4E8532C65B
:10410000EFF05FE9B3068A0083C7E6FF83C6F6FFD8
:104110003246A207D58F6315F500D947638FFD029C
:104120000D47A68763F3E4008D4793F4F70FBDB7FF
:104130006949014B9305D9FF93F5F50F4E85EFF0D3
:104140007FE583477A0183468A01A207D58FE399E9
:10415000A7FCD947E396FDFC4A8693858A805E8555
:10416000EFF03FE7BDBFE947E304F6FC014B6949C7
:10417000BDB7A947E300F6F4E3080BF6B147054BDA
:10418000E314F6F60349BA0006093D093284E9B59D
:1041900058218547631BF700EFC2AFA0503193054C
:1041A00065000841A9266FC00FA28280EFC26F9FF1
:1041B000376500001305C55DEFD04F9003A5418C16
:1041C000EFF09FE413054006EFD0DFA1C5BFEFC2BB
:1041D0004F9D3765000059711305055FEFD00F8EB5
:1041E000376400001306400681456800EFC06F9EEB
:1041F00003A5018BFD56130640066C00EFC07F84BB
:104200001305C45FEFD08F8B6800EFF07FF8D9BF44
:10421000EFC22F99B745000037650000D147094725
:104220009306002001469385C51A1305455DEFD01E
:104230005F8919C1EFD0BFA06FC0EF98EFC26F9632
:10424000B745000037650000D1470D4793060020B1
:1042500001469385E51C1305855EEFD09F8619C145
:10426000EFD0FF9D6FC02F96EFC2AF933765000070
:1042700081461546930520031305C560EFC04FEC3A
:1042800023A8A18A3335A0006FC0EF9311CD1C2164
:1042900089CFEFC20F91484193F5F50FEF003049F8
:1042A00085473E856FC02F9281473E858280EFC251
:1042B0004F8F2A845C400965130505583727004055
:1042C00008C4930607806396D700EF0090036FC081
:1042D0008F8F930607C06395D700EF001006C5BF08
:1042E000B7460040938606406395D700EF007008FC
:1042F000F9BF6395E700EF00500BD1BF375700407F
:1043000013070780E395E7FCEF00D0235C4C81E7BF
:10431000EF00B01F6DBF15476395E700EF00B032A7
:104320007DB719476395E700EF0090354DB71D47FE
:104330006395E700EF00703859BF21476395E700A8
:10434000EF00503B69B72547E393E7F8EF003017DC
:10435000BDBFEFC20F85B704002013848417B725B3
:10436000002013060008938585851305C400EFE03F
:104370005FF513858417EFF09FF3B7250020854480
:10438000130600089385858D1305C40223AA818A2C
:104390001309040204A0EFE0DFF24A85EFF03FF1D9
:1043A000B725002013060008938585951305C404DE
:1043B00023AC218B2300940213090404EFE07FF067
:1043C0004A85EFF0DFEEB72500201306000893853D
:1043D000859D1305C40623AE218B23009404130985
:1043E0000406EFE01FEE4A85EFF07FECB7250020D2
:1043F00013060008938585A51305C40823A0218D05
:104400002300940613090408EFE0BFEB4A85EFF0A0
:104410001FEAB725002013060008938585AD130514
:10442000C40A23A2218D230094081309040AEFE093
:104430005FE94A85EFF0BFE72300940A23A4218DAA
:1044400001456FB05FF8EFB2DFF585451145EFE04C
:10445000BFCE6FB05FF7EFB2DFF481451145EFE0FB
:10446000BFCD6FB05FF6EFB2DFF385451545EFE0E6
:10447000BFCC6FB05FF5EFB2DFF281451545EFE0DD
:10448000BFCB6FB05FF4EFB2DFF185456145EFE080
:10449000BFCA6FB05FF3EFB2DFF081456145EFE077
:1044A000BFC96FB05FF2EFB2DFEF85451305300291
:1044B000EFE09FC86FB03FF1EFB2BFEE814513054B
:1044C0003002EFE07FC76FB01FF0EFB29FED854580
:1044D00013057003EFE05FC66FB0FFEEEFB27FEC45
:1044E000814513057003EFE03FC56FB0DFEDEFB21C
:1044F000BFE903A7418B2A842E8AB2891389418B95
:10450000631FA700EFF03FF4814463C6340583279F
:104510000900639B8704EFF01FF46FB03FEA83A7A5
:10452000818B6395A700EFF01FF4F9BF83A7C18BC0
:104530006395A700EFF03FF5C1BF83A7018C63959A
:10454000A700EFF05FF6C9B783A7418CE39EA7FAF7
:10455000EFF0BFF755BFB3079A00838507002285A8
:104560008504EFF0BFD255B783A7818B6395870091
:10457000EFF07FF05DB783A7C18B63958700EFF005
:104580009FF161BF83A7018C63958700EFF0DFF295
:1045900069B783A7418CE39287F8EFF03FF4B5BF8A
:1045A000814709C91821814711C75C49084D898F86
:1045B000B337F0003E858280EFB2BFDE41112A841E
:1045C000A3070100EFF0DFFD19C59305F100130506
:1045D000C400EFE0DFD20305F10041016FB0BFDEA0
:1045E000EFB23FDC3105EFE0FFD36FB0DFDDB7F7AF
:1045F000FF1F03A5477082805841032805004C45E2
:1046000037060140930706403E979346F8FFB1C531
:1046100083250640F58D2320B640D043F18ED4C3C8
:104620001443B3E6060114C3184190479346F7FFBD
:10463000758E90C7D047F18ED4C714454146639913
:10464000C6009447D98E94C7D447558FD8C7828067
:10465000B6979443558F98C382801C43F58F1CC333
:104660008280B70701401387074083A70740584B54
:10467000698F09C77D8D3335A00082800145828016
:10468000B707014023AAA74082809C4513F7070182
:1046900013F8F70001C7D8413368E8008E2113F7FB
:1046A000F50F39C318418146854E3D4F930F800267
:1046B00093028004214E3396DE00B3F8C5006311E7
:1046C00016039398260033131F011343F3FF337728
:1046D000E300B318180133E7E800639FF70550C9FA
:1046E0008506E39AC6FD18C11307F00F6375B7047A
:1046F00054412146854E3D4F930F80029302800422
:10470000414EB398CE0033F715016392E8021317B8
:10471000260001173313EF001343F3FFB376D300E2
:104720003317E800D98E639DF701232A150105068A
:10473000E319C6FD54C18280E39457FA10C94DB7FE
:10474000E39757FE23281501DDB708456D8D3335F6
:10475000A000828019C20CC982804CC9828013F7E4
:10476000C50F93F73500B7050140BA9594458A0700
:104770003D473317F7001347F7FF758F98C59845E6
:104780003315F500598D88C5828003A7C18C8947F0
:1047900010216311F70214318D4763EDD7003C21DE
:1047A0009A0637E700E09607D58F93F7F70F329711
:1047B0002300F74054410547935756003317C7006D
:1047C00089CA938707048A07B7E600E0B69798C3BB
:1047D000828093870706C5BF371702405C43914626
:1047E000B18B6385D700A1466382D706B7177A00DD
:1047F000938707201CC1371602405C423707002010
:10480000130787239183BD8BBA9794231C41B3D799
:10481000D7005CC15442A1829D8ABA969422B3D635
:10482000D70014C55442AD829D8A36971823B3D75A
:10483000E7005CC55842398393763700138741807F
:1048400036971823B3D7E7021CC982805C435843CC
:10485000C166C983758FB7F6FF1F83A6C670BD8B6F
:1048600089071396160163480600C5460146639200
:10487000D702C94739A88946638FD702BD46638EE0
:10488000D702C146638ED702C54601466393D7005F
:10489000C1471DEF3747024003270780418B05C7FB
:1048A00037177A0013070720B307F7021CC121D678
:1048B0001C41858381B701466DBF0546B547D1BF11
:1048C0000146BD47F9B737173D0013070790E9BF09
:1048D000B7150240D8559316F700D85563DF060484
:1048E00011833D8B9306170037177A0013070720B3
:1048F0003357D70218C1D455A182BD8A8DE295469F
:104900003307D702058318C137170240585714419F
:104910003D8B050733D7E60218C1184171B78545AD
:104920006394B600E546E9BFBD456396B600D1463F
:104930003387E602C9BF8906E5BF3D8B93061700A2
:1049400037177A00130707203357D702F1B799C5F5
:10495000371702401C4F5D8D08CF8280B717024089
:10496000984F1345F5FF798D88CF828099C5371709
:1049700002405C4F5D8D48CF8280B7170240D84F10
:104980001345F5FF798DC8CF8280EFB29FA116291C
:10499000F577FD17F58FF621DA257971D58F1EA9E8
:1049A0005625FD779387379FF58FD6212A842EC60B
:1049B000D58F9625D58FB625D58F5EA55E29C207E2
:1049C000C18393F7F7CFD98F5EA96808EFF0DFE0D6
:1049D000B747014093870780B245631EF402A25790
:1049E0006547B387E7029841930640060A07B3D7A5
:1049F000E70233D7D702B3F7D7021207920793879C
:104A00002703B3D7D702BD8BD98FC207C1831EA49A
:104A100045616FB05F9B9257E1B791C55E2509670D
:104A2000D98F5EA582805A25F977FD17F98FD5BFFA
:104A300013F7F50F85471583B395B7006319F70092
:104A40009307C500984301CED98D8CC382808946D7
:104A500093074501E318D7FE93070501E5B793C512
:104A6000F5FFF98DDDB793F5F51F4EA182804A2140
:104A70001375F51F82800A216D8D3335A000828069
:104A800013F7F50F85461583B397B6006311D70268
:104A90005A25F98F1A2101454207418381CB0545EB
:104AA000A181B315B5006D8F3335E0008280894652
:104AB0006314D7001A29F1BF5A29E1BFA1818547A4
:104AC000B397B70093C7F7FFC207C1831EA18280C7
:104AD000EFB23F8D81450945EFE06FE46FB0BF8EC7
:104AE000EFB23F8C85450945EFE00FE56FB0BF8D14
:104AF000EFB23F8B854513056002EFE0EFE36FB047
:104B00009F8CEFB21F8A81451145EFE04FE181454F
:104B10001145EFE06FE2814513056002EFE02FE001
:104B2000EFF01FFD6FB03F8AEFB2BF8785451305D9
:104B30007002EFE06FE06FB01F89EFB29F86814592
:104B40001545EFE0CFDD81451545EFE0EFDE81450E
:104B500013057002EFE0AFDCEFF01FFD6FB0BF8612
:104B6000EFB23F84854513058002EFE0EFDC6FB0C4
:104B70009F85EFB21F8381456145EFE04FDA8145A4
:104B80006145EFE06FDB814513058002EFE02FD92F
:104B9000EFF01FFD6FB03F83EFB2BF808545130577
:104BA0009002EFE06FD96FB01F82EFB28FFF8145A7
:104BB00013053002EFE0AFD6814513053002EFE078
:104BC000AFD7814513059002EFE06FD5EFF0DFFC22
:104BD0006FB06FFF411122C6375400409305505209
:104BE00013050480EFF0DFE915C513050480EFF02D
:104BF0001FE89375F50F2388B18C03A5418C1C4DDC
:104C0000104954498507B3E7C7026385D7003105CA
:104C1000EFE02FEC3244410173002030EFB26FF827
:104C200085451305A002EFE02FD16FB0CFF9EFB2A9
:104C30004FF781451305A002EFE00FD06FB0AFF83A
:104C4000EFB22FF685451305B002EFE0EFCE6FB05F
:104C50008FF7EFB20FF581451305B002EFE0CFCD2E
:104C60006FB06FF6EFB2EFF385451305C002EFE0CA
:104C7000AFCC6FB04FF5EFB2CFF281451305C00254
:104C8000EFE08FCB6FB02FF4EFB2AFF18545130596
:104C9000D002EFE06FCA6FB00FF3EFB28FF0814533
:104CA0001305D002EFE04FC96FB0EFF1EFB26FEF35
:104CB00085451305E002EFE02FC86FB0CFF0EFB2EB
:104CC0004FEEEFF0DFF6EFF0DFF8EFF0DFFAEFF0A6
:104CD000DFFCEFF0BFFD854513058003EFE0CFC596
:104CE000814513059003EFE02FC585451305A0030B
:104CF000EFE08FC46FB02FEDEFB2AFEA814513053F
:104D0000E002EFE06FC36FB00FECEFB28FE9EFF0AE
:104D10001FF2EFF01FF4EFF01FF6EFF01FF8EFF0C7
:104D2000BFFD814513058003EFE00FC181451305E9
:104D30009003EFE06FC081451305A003EFE0CFBF04
:104D40006FB06FE8EFB2EFE57971AA848145130582
:104D5000A002EFE0CFBC81451305B002EFE02FBC0D
:104D600081451305C002EFE08FBB81451305D002DA
:104D7000EFE0EFBA81451305E002EFE04FBA81455D
:104D800013057003EFE0AFB9814513057003EFE041
:104D9000AFBA814513058003EFE06FB88145130575
:104DA0009003EFE0CFB781451305A003EFE02FB7E5
:104DB000EFF0BFF585452145EFF07FB98545370513
:104DC0000400EFF0BFBA93070040FC8237140140A3
:104DD0008D473ECC4C08E147130504C03ECEEFF0B2
:104DE000DF8A856793870780FC824C08914713050B
:104DF00004C03ECE37540040EFF03F890C10B70797
:104E00000C001305048026D03ED402D223160102E2
:104E1000EFF0BFB7930770137C8685475C87680007
:104E200085473EC8EFF07F9605461305048093053D
:104E30005052EFF0FFBF854513050480EFF0FFBD32
:104E400045616FB04FD8EFB2CFD5EFF03FDDEFF057
:104E50005FE0EFF05FE2EFF05FE4EFF0FFE9814544
:104E600013058003EFE04FAD814513059003EFE09C
:104E7000AFAC81451305A003EFE00FAC6FB0AFD42A
:104E8000EFB22FD2EFF0BFDAEFF09FDBEFF0BFDE33
:104E9000EFF0BFE0EFF05FE6854513058003EFE03C
:104EA000AFA9814513059003EFE00FA981451305D4
:104EB000A003EFE06FA86FB00FD1EFB28FCEEFF08D
:104EC0001FD7EFF01FD9EFF0FFD9EFF01FDDEFF0A4
:104ED000BFE2854513058003EFE00FA68545130566
:104EE0009003EFE06FA581451305A003EFE0CFA489
:104EF0006FB06FCDEFB2EFCAEFF07FD3EFF07FD599
:104F0000EFF07FD7EFF05FD8EFF01FDF814513059B
:104F10008003EFE06FA2814513059003EFE0CFA17E
:104F200085451305A003EFE02FA16FB0CFC9EFB205
:104F30004FC72A84EFF03FB3930500082285EFF0B6
:104F40009FB37DD96FB02FC801476314E6000145B8
:104F50008280B307E5000507B386E5009C2383C67E
:104F6000F6FFE384D7FE3385D7408280B3C7A50020
:104F70008D8B3307C50081E78D4763EDC700AA8796
:104F8000637EE508942185078505A38FD7FEE3EBB3
:104F9000E7FE828093763500AA8789CA9421850727
:104FA0008505A38FD7FE93F63700C5BF9376C7FF5D
:104FB000138606FE63F0C70683A3050083A245009F
:104FC00083AF850003AFC50083AE050103AE450185
:104FD00003A3850183A8C5019385450223A077001B
:104FE00003A8C5FF23A2570023A4F70123A6E701C6
:104FF00023A8D70123AAC70123AC670023AE17015A
:105000009387470223AE07FF75B79041910791053B
:1050100023AEC7FEE3EBD7FEE3E6E7F68280AA877E
:1050200098239386170009EB850503C7F5FF8507CD
:10503000A38FE7FE75FB8280B687DDB7AA8798212C
:1050400085078505A38FE7FE7DFB8280AA878507FC
:1050500003C7F7FF6DFF3385A7407D15828015C21A
:105060007D160147B307E500B386E5009C23942233
:105070006396D7006304C7000507EDF73385D74073
:105080008280014582800000505B0000645B00006C
:10509000745B0000885B0000945B0000A05B000074
:1050A000A45B0000B45B0000C45B0000CC5B0000AC
:1050B000E05B0000F05B0000F85B0000045C0000B7
:1050C000105C0000245C00002C5C00003C5C0000D4
:1050D0004C5C0000645C00006D61696E00000000C3
:1050E000546F20696E697469616C697A65206465C2
:1050F000766963653A2573206661696C65642E2064
:10510000546865206572726F7220636F64652069F0
:10511000732025640A0000007469646C6500000057
:105120000000010002000100030001000200010074
:105130000400010002000100030001000200010060
:10514000050001000200010003000100020001004F
:105150000400010002000100030001000200010040
:10516000060001000200010003000100020001002E
:105170000400010002000100030001000200010020
:10518000050001000200010003000100020001000F
:105190000400010002000100030001000200010000
:1051A00007000100020001000300010002000100ED
:1051B00004000100020001000300010002000100E0
:1051C00005000100020001000300010002000100CF
:1051D00004000100020001000300010002000100C0
:1051E00006000100020001000300010002000100AE
:1051F00004000100020001000300010002000100A0
:10520000050001000200010003000100020001008E
:10521000040001000200010003000100020001007F
:1052200030313233343536373839414243444546DC
:10523000000000000A205C207C202F0A00000000F3
:105240002D205254202D202020202054687265618A
:1052500064204F7065726174696E6720537973744E
:10526000656D0A004A756C203137203230323400C7
:10527000202F207C205C202020202025642E2564E7
:105280002E2564206275696C642025730A00000075
:105290002032303036202D203230313920436F70AB
:1052A0007972696768742062792072742D746872EB
:1052B000656164207465616D0A000000284E554CDC
:1052C0004C29000030313233343536373839616299
:1052D0006364656600000000746F74616C206D6526
:1052E0006D6F72793A2025640A0000007573656459
:1052F000206D656D6F7279203A2025640A000000E8
:105300006D6178696D756D20616C6C6F636174653A
:1053100064206D656D6F72793A2025640A00000083
:105320006C697374206D656D6F7279207573616738
:105330006520696E666F726D6174696F6E00000042
:105340006C6973745F6D656D00000000746F20669A
:10535000726565206120626164206461746120620D
:105360006C6F636B3A0A00006D656D3A20307825EA
:105370003038782C207573656420666C61673A203C
:1053800025642C206D6167696320636F64653A2032
:105390003078253034780A006865617000000000BC
:1053A0006D656D20696E69742C206572726F722054
:1053B000626567696E20616464726573732030781A
:1053C00025782C20616E6420656E642061646472AF
:1053D00065737320307825780A0000001B5B324A21
:1053E0001B5B48002D2D46756E6374696F6E204CF3
:1053F0006973743A0A0000005F5F0000252D3136A2
:1054000073202D2D2025730A000000006465766945
:1054100063650000252D2A2E7320202020202020C7
:1054200020207479706520202020202020202072E8
:10543000656620636F756E740A000000202D2D2DA7
:105440002D2D2D2D2D2D2D2D2D2D2D2D2D2D2D2D8C
:105450002D202D2D2D2D2D2D2D2D2D2D0A00000033
:10546000252D2A2E2A7320252D32307320252D3804
:10547000640A00006576656E74000000252D2A2EF2
:105480007320202020202073657420202020737535
:105490007370656E64207468726561640A00000050
:1054A00020202D2D2D2D2D2D2D2D2D2D202D2D2D53
:1054B0002D2D2D2D2D2D2D2D2D2D2D0A00000000F3
:1054C000252D2A2E2A732020307825303878202563
:1054D0003033643A00000000252D2A2E2A73202044
:1054E00030782530387820300A0000006D61696C12
:1054F000626F7800252D2A2E7320656E74727920D4
:1055000073697A652073757370656E642074687250
:105510006561640A00000000202D2D2D2D20202D16
:105520002D2D2D202D2D2D2D2D2D2D2D2D2D2D2DB8
:105530002D2D0A00252D2A2E2A7320253034642093
:1055400020253034642025643A000000252D2A2EC1
:105550002A732025303464202025303464202564CB
:105560000A0000006D7367717565756500000000C5
:10557000252D2A2E7320656E7472792073757370D1
:10558000656E64207468726561640A00202D2D2D9B
:105590002D20202D2D2D2D2D2D2D2D2D2D2D2D2D55
:1055A0002D0A0000252D2A2E2A7320253034642050
:1055B0002025643A00000000252D2A2E2A7320257C
:1055C000303464202025640A000000006D75746585
:1055D00078000000252D2A2E732020206F776E651D
:1055E000722020686F6C642073757370656E642020
:1055F0007468726561640A00202D2D2D2D2D2D2DCE
:105600002D202D2D2D2D202D2D2D2D2D2D2D2D2DE4
:105610002D2D2D2D2D0A0000252D2A2E2A73202513
:105620002D382E2A7320253034642025640A00008A
:1056300073656D6170686F7265000000252D2A2EFC
:1056400073207620202073757370656E64207468F3
:10565000726561640A000000202D2D2D202D2D2D56
:105660002D2D2D2D2D2D2D2D2D2D2D0A0000000041
:10567000252D2A2E2A7320253033642025643A00F4
:10568000252D2A2E2A7320253033642025640A0014
:105690007468726561640000252D2A2E7320707273
:1056A000692020737461747573202020202020737A
:1056B000702020202020737461636B2073697A65E9
:1056C000206D61782075736564206C656674207444
:1056D00069636B20206572726F720A00202D2D2D78
:1056E00020202D2D2D2D2D2D2D202D2D2D2D2D2D11
:1056F0002D2D2D2D202D2D2D2D2D2D2D2D2D2D20F4
:10570000202D2D2D2D2D2D20202D2D2D2D2D2D2DF0
:105710002D2D2D202D2D2D0A00000000252D2A2EA7
:105720002A7320253364200020726561647920206B
:10573000000000002073757370656E640000000047
:1057400020696E69742020200000000020636C6FC7
:105750007365202000000000203078253038782044
:1057600030782530387820202020253032642525D7
:1057700020202030782530387820253033640A0006
:1057800074696D6572000000252D2A2E732020702B
:105790006572696F64696320202074696D656F7537
:1057A0007420202020202020666C61670A00000001
:1057B000202D2D2D2D2D2D2D2D2D2D202D2D2D2D33
:1057C0002D2D2D2D2D2D202D2D2D2D2D2D2D2D2D16
:1057D0002D2D0A00252D2A2E2A73203078253038C9
:1057E00078203078253038782000000061637469B3
:1057F00076617465640A000064656163746976614A
:105800007465640A0000000063757272656E74202E
:105810007469636B3A3078253038780A00000000EC
:105820006C69737420616C6C2073796D626F6C208D
:10583000696E2073797374656D0000006C69737410
:10584000000000006C6973742064657669636520EC
:10585000696E2073797374656D0000005F5F636D1E
:10586000645F6C6973745F646576696365000000EA
:105870006C6973742064657669636520696E207352
:10588000797374656D0000006C6973745F6465768C
:10589000696365006C6973742074696D6572206951
:1058A0006E2073797374656D000000005F5F636D37
:1058B000645F6C6973745F74696D657200000000E9
:1058C0006C6973742074696D657220696E207379D8
:1058D0007374656D000000006C6973745F74696DAA
:1058E000657200006C697374206D65737361676520
:1058F00020717565756520696E2073797374656DA7
:10590000000000005F5F636D645F6C6973745F6DBE
:1059100073677175657565006C697374206D657367
:105920007361676520717565756520696E2073798F
:105930007374656D000000006C6973745F6D73674C
:1059400071756575650000006C697374206D61691F
:105950006C20626F7820696E2073797374656D00B6
:105960005F5F636D645F6C6973745F6D61696C62C6
:105970006F7800006C697374206D61696C20626FD0
:105980007820696E2073797374656D006C69737427
:105990005F6D61696C626F78000000006C69737400
:1059A000206D7574657820696E2073797374656DE8
:1059B000000000005F5F636D645F6C6973745F6D0E
:1059C00075746578000000006C697374206D7574DF
:1059D000657820696E2073797374656D000000002E
:1059E0006C6973745F6D7574657800006C697374AD
:1059F000206576656E7420696E2073797374656DA9
:105A0000000000005F5F636D645F6C6973745F65C5
:105A100076656E74000000006C69737420657665AD
:105A20006E7420696E2073797374656D00000000D8
:105A30006C6973745F6576656E7400006C6973746D
:105A40002073656D6170686F726520696E2073796F
:105A50007374656D000000005F5F636D645F6C6967
:105A600073745F73656D00006C6973742073656D8A
:105A70006170686F6E6520696E2073797374656DEF
:105A8000000000006C6973745F73656D00000000B6
:105A90006C69737420746872656164005F5F636D24
:105AA000645F6C6973745F746872656164000000A0
:105AB0006C69737420746872656164006C697374D6
:105AC0005F74687265616400746865207465726DE6
:105AD000696E616C2073637265656E005F5F636DF4
:105AE000645F636C65617200746865207465726DD3
:105AF000696E616C2073637265656E00636C6561CD
:105B0000720000007265626F6F74207468652062B5
:105B10006F617264000000005F5F636D645F7265B7
:105B2000626F6F74000000007265626F6F742074A2
:105B3000686520626F617264000000007265626FC8
:105B40006F7400002D000000257300002F0000007E
:105B50004368617261637465722044657669636548
:105B600000000000426C6F636B20446576696365DA
:105B7000000000004E6574776F726B20496E74658B
:105B800072666163650000004D5444204465766987
:105B90006365000043414E204465766963650000FB
:105BA00052544300536F756E642044657669636593
:105BB000000000004772617068696320446576697F
:105BC00063650000493243204275730055534220FB
:105BD000536C61766520446576696365000000005A
:105BE00055534220486F73742042757300000000C3
:105BF00053504920427573005350492044657669DB
:105C0000636500005344494F204275730000000053
:105C1000504D2050736575646F20446576696365E7
:105C2000000000005069706500000000506F727441
:105C3000616C2044657669636500000054696D6598
:105C40007220446576696365000000004D697363E6
:105C5000656C6C616E656F7573204465766963650C
:105C600000000000556E6B6E6F776E00546F6F20F2
:105C70006D616E7920617267732021205765206FF6
:105C80006E6C79205573653A0A0000002573200078
:105C900025733A20636F6D6D616E64206E6F7420A2
:105CA000666F756E642E0A0052542D5468726561D9
:105CB00064207368656C6C20636F6D6D616E6473D6
:105CC0003A0A00005F5F636D645F0000252D313686
:105CD00073202D2025730A0052542D54687265617B
:105CE00064207368656C6C2068656C70000000004F
:105CF0005F5F636D645F68656C70000053686F7709
:105D000020746865206D656D6F72792075736167A9
:105D10006520696E207468652073797374656D0001
:105D20005F5F636D645F6672656500004C697374E4
:105D3000207468726561647320696E2074686520E0
:105D400073797374656D00005F5F636D645F70737A
:105D5000000000006D7368200000000066696E732B
:105D6000682000003E00000066696E73683A206398
:105D7000616E206E6F742066696E6420646576695A
:105D800063653A2025730A006E6F206D656D6F7232
:105D90007920666F72207368656C6C0A00000000E1
:105DA000747368656C6C00007368727800000000A2
:105DB000080000002563000008257320200800006B
:105DC000082008001B5B324B0D0000002573257373
:105DD0000000000072656164207374617475732043
:105DE00066726F6D20686172647761726520706998
:105DF0006E00000070696E526561640077726974AC
:105E0000652076616C756520746F206861726477B7
:105E10006172652070696E0070696E577269746591
:105E200000000000736574206861726477617265B8
:105E30002070696E206D6F646500000070696E4DA2
:105E40006F646500756172743100000020340000D9
:105E5000E0330000023400009E34000030350000C2
:105E60008A3500000100000016000000020000005A
:105E700017000000040000001800000008000000E7
:105E800019000000100000001A00000020000000AF
:105E900027000000400000002700000080000000F4
:105EA00027000000000100002700000000020000A1
:105EB0002700000000040000380000000008000077
:105EC0003800000000100000380000000020000032
:105ED0003800000000400000380000000080000092
:105EE00038000000FFFFFFFF00000000000000007E
:105EF0000000000001000000923300000018014083
:105F0000040000000200000092330000001801406D
:105F10000800000003000000923300000018014058
:105F2000100000000400000092330000001801403F
:105F3000200000000500000092330000001801401E
:105F400040000000FFFFFFFF000000000000000015
:105F50000000000007000000823300000010014034
:105F60000020000008000000823300000010014003
:105F700000400000090000008233000000100140D2
:105F800000800000FFFFFFFF000000000000000095
:105F900000000000FFFFFFFF000000000000000005
:105FA00000000000FFFFFFFF0000000000000000F5
:105FB00000000000FFFFFFFF0000000000000000E5
:105FC00000000000FFFFFFFF0000000000000000D5
:105FD000000000000F0000008233000000100140AC
:105FE000010000001000000082330000001001409A
:105FF0000200000011000000823300000010014088
:106000000400000012000000823300000010014074
:1060100008000000FFFFFFFF00000000000000007C
:1060200000000000FFFFFFFF000000000000000074
:1060300000000000FFFFFFFF000000000000000064
:1060400000000000FFFFFFFF000000000000000054
:10605000000000001700000072330000000801403B
:106060000100000018000000723300000008014029
:106070000200000019000000723300000008014017
:10608000040000001A000000723300000008014004
:1060900008000000FFFFFFFF0000000000000000FC
:1060A00000000000FFFFFFFF0000000000000000F4
:1060B000000000001D0000007233000000080140D5
:1060C000100000001E0000007233000000080140B4
:1060D000200000001F000000723300000008014093
:1060E0004000000020000000723300000008014062
:1060F00080000000210000008233000000100140F9
:106100001000000022000000823300000010014057
:10611000200000002300000062330000000C01405A
:10612000010000002400000062330000000C014068
:10613000020000002500000062330000000C014056
:106140000400000026000000923300000018014007
:10615000800000002700000092330000001801407A
:1061600000010000280000009233000000180140E8
:1061700000020000290000009233000000180140D6
:10618000000400002A0000009233000000180140C3
:10619000000800002B0000009233000000180140AE
:1061A000001000002C000000923300000018014095
:1061B000002000002D000000923300000018014074
:1061C000004000002E000000923300000018014043
:1061D000008000002F00000062330000000C01402E
:1061E000000400003000000062330000000C014099
:1061F00000080000FFFFFFFF00000000000000009B
:1062000000000000FFFFFFFF000000000000000092
:10621000000000003300000062330000000C014069
:10622000001000003400000062330000000C014048
:10623000002000003500000062330000000C014027
:10624000004000003600000062330000000C0140F6
:1062500000800000370000005033000000140140AF
:10626000000100003800000050330000001401401D
:10627000000200003900000050330000001401400B
:10628000000400003A0000005033000000140140F8
:10629000000800003B0000005033000000140140E3
:1062A000001000003C0000005033000000140140CA
:1062B000002000003D0000005033000000140140A9
:1062C000004000003E000000503300000014014078
:1062D000008000003F0000008233000000100140F9
:1062E0004000000040000000823300000010014028
:1062F00080000000410000008233000000100140D7
:106300000001000042000000823300000010014044
:10631000000200004300000072330000000801404A
:10632000000100004400000072330000000801403A
:106330000002000045000000723300000008014028
:106340000004000046000000723300000008014015
:106350000008000047000000723300000008014000
:1063600000100000480000007233000000080140E7
:1063700000200000FFFFFFFF000000000000000001
:1063800000000000FFFFFFFF000000000000000011
:1063900000000000FFFFFFFF000000000000000001
:1063A000000000004C0000007233000000080140B3
:1063B000004000004D000000723300000008014062
:1063C000008000004E0000008233000000100140F9
:1063D000000400004F000000823300000010014064
:1063E000000800005000000082330000001001404F
:1063F0000010000051000000503300000014014064
:106400000100000052000000503300000014014061
:10641000020000005300000050330000001401404F
:10642000040000005400000050330000001401403C
:106430000800000055000000503300000014014027
:10644000100000005600000050330000001401400E
:1064500020000000570000005033000000140140ED
:1064600040000000580000005033000000140140BC
:10647000800000005900000062330000000C014061
:10648000080000005A00000062330000000C0140C8
:10649000100000005B00000062330000000C0140AF
:1064A000200000005C00000062330000000C01408E
:1064B000400000005D00000062330000000C01405D
:1064C00080000000FFFFFFFF000000000000000050
:1064D000000000005F00000062330000000C01407B
:1064E000000100006000000062330000000C014069
:1064F000000200006100000092330000001801401B
:10650000010000006200000092330000001801400A
:1065100002000000FFFFFFFF00000000000000007D
:1065200000000000FFFFFFFF00000000000000006F
:106530000000000070696E00CE380000A43A000030
:10654000823A0000603A0000CA3800002068617298
:106550006466756C740D0A00204E4D492048616ECA
:10656000646C65720D0A00000D0A204D43553A20F7
:1065700043483332563330330D0A000020537973C9
:10658000436C6B3A202564487A0D0A002043686901
:106590007049443A20253038780D0A0072745F6DD6
:1065A000715F73656E64204552520A0072745F6DAC
:1065B000715F73656E640A0072696E675F717565FD
:1065C00075655F6C656E677468203D202564200AE0
:1065D0000000000052656376000000000A2052654A
:1065E0006376200A0000000073656E6400000000FE
:1065F0000A2053656E64200A000000000A205365DB
:106600006E642062756666200A00000053656E6441
:106610005F6D71004053000020530000081400001B
:106620003C58000020580000022500005C58000083
:1066300044580000D423000088580000705800001F
:10664000D4230000AC5800009458000068240000D7
:10665000D8580000C0580000682400000459000009
:10666000E45800001E2300003859000018590000AB
:106670001E230000605900004859000060220000FD
:106680008C5900007459000060220000B4590000C9
:106690009C590000DE210000E0590000C8590000AC
:1066A000DE210000045A0000EC59000032210000F5
:1066B000305A0000185A000032210000585A0000D9
:1066C0003C5A00007C200000845A0000685A0000F8
:1066D0007C2000009C5A0000905A0000981F000087
:1066E000BC5A0000B05A0000981F0000DC5A00009D
:1066F000C85A0000EE1E0000FC5A0000E85A0000D4
:10670000EE1E0000185B0000045B0000DC1E0000B1
:106710003C5B0000285B0000DC1E0000F05C000019
:10672000D85C00004C250000205D0000FC5C0000EF
:1067300002280000485D00002C5D0000F4270000E6
:10674000F45D0000D45D000052310000185E0000CE
:10675000FC5D0000383100003C5E0000245E00005B
:106760001E310000D0040000D8040000A433000053
:106770009C390000DC04000022280000D404000042
:106780000100000004000020040000208000000040
:10679000020000001400002014000020200000006F
:1067A000030000002400002024000020240000003A
:1067B000040000003400002034000020200000000D
:1067C00005000000440000204400002030000000CC
:1067D0000600000054000020540000203400000097
:1067E0000900000064000020640000204400000054
:1067F0000A00000074000020740000202C0000003B
:10680000FFFF00000000000000000000FFFF00008C
:106810000000000000000000FFFF0000000000007A
:1068200000000000FFFF000000000000000000006A
:10683000FFFF00000000000000000000FFFF00005C
:106840000000000000000000FFFF0000000000004A
:1068500000000000FFFF000000000000000000003A
:10686000FFFF00000000000000000000FFFF00002C
:106870000000000000000000FFFF0000000000001A
:1068800000000000FFFF000000000000000000000A
:10689000FFFF00000000000000000000FFFF0000FC
:1068A0000000000000000000FFFF000000000000EA
:1068B00000000000FFFF00000000000000000000DA
:1068C00000000000000000000102030406070809A0
:1068D000300000002E3F0000A1000000B83E000084
:1068E000534C0000000000000016000000000000F3
:1068F0000000000000000000000000000018004040
:106900000000000000000000000000000000000087
:10691000000000000100000000000000001C00401A
:106920000000000000000000000000000000000067
:1069300000000000010000000000000000440040D2
:106940000000000000000000000000000000000047
:1069500000000000010000000000000000200040D6
:106960000000000000000000000000000000000027
:10697000000000000100000000000000004800408E
:106980000000000000000000000000000000000007
:106990000000000000000000000000000050004067
:1069A00000000000000000000000000000000000E7
:1069B00000000000010000000000000001020304CC
:1069C000010203040607080900D8B80502040608F6
:00000001FF
